:020000040030CA
:0E00000000C80F000080800003C003A0034072
:020000040000FA
:020000001FD00F
:020000040000FA
:02000800FFD027
:020000040000FA
:02001800FFD017
:020000040000FA
:10004000CBD09EBA01D0FDD7ABA203D0AB98AB8882
:10005000F8D7EC6EAE50ABA402D0ED50F2D7120040
:10006000ACB201D0FDD7AD6EED5012000500E9DF56
:10007000FD6EED50E6DFFE6EED501200EC6E000EF0
:10008000EFD7A68EA69C88D8F9D7A68EA69C87D82F
:10009000F5D70F0B8DD812000ED0E2D70ED041D07D
:1000A00047D0ECD7FF0019D00DD02CD020D047D0AE
:1000B00033D0E7D7EAD7C5DFE1D7D8DFDFD7C1DF55
:1000C000E8DFFDD7BEDFE46EED50EC6E0900F550C1
:1000D000C7DFE706FAE1E5521200B3DFE46EED5048
:1000E000EC6EDE50BDDFE706FBE1E5521200A9DF52
:1000F000E46EED50A6DFF56E0D00ED50E706FAE177
:10010000E552BCD79EDFE46EED509BDFDE6EED5016
:10011000E706FBE1E552B2D75BD8EC6E0800F528A4
:10012000D2D78FDF8EDFDA6EED50D96EED50A6D7C5
:1001300088DF87DFF76EED50F66EED509FD7EC6EDF
:10014000400EE46EFF0EEC6E0900F550ED14E7066C
:10015000FAE1E55285D7EC6EFD50F66EFE50F76E73
:10016000ED5006001200D96E800AE834DA50DA5AEF
:10017000ED501200F8DFEC6EDE501200F4DFDE6EA0
:10018000ED501200EC6EF29E550EA76EAA0EA76EF1
:10019000A682F28EED501200A684A688F3D7A6841C
:1001A000A6980A00EFDF09001200EF60EF6EED5035
:1001B000E844FD26010BFE22ED50120000EE7FF018
:1001C00010EE8FF08A68EC6E700ED36EED50120058
:1001D000C2DF057069633138000EFC6EEFDFC18A43
:1001E000C18C93889382EC6E330EAF6E240EAC6E8E
:0E01F000900EAB6EED5081A801D061D701D00A
:020000040000FA
:10024000EF36E8340500FE6EED50FD6EED50120005
:10025000DA6AD96EFD50DE6EFE50DE6EED5006009D
:100260001200E844FD26010BFE22FD90FD50F66EC3
:10027000FE50F76EED500600EC6E0900F550EC6E86
:100280000900F5501200EC6E000EEC6E080EE46EE4
:10029000ED50D8901336143606E3EC6E1550131A51
:1002A0001650141AED50E834E706F3E1E552120057
:1002B000EC6E000EEC6E010EEADF14501200EC6ED4
:1002C000D650090F0424EC6E0550D722ED50D66E9F
:1002D000ED501200EC6ECE50070F0624EC6E075066
:1002E000CF22ED50CE6EED501200EC6EB250070FE3
:1002F0000824EC6E0950B322ED50B26EED5012009E
:10030000EC6E0550D76E0450D66EED501200EC6EB8
:100310000750CF6E0650CE6EED501200EC6E0950B5
:10032000B36E0850B26EED5012001DD80DA003D070
:100330008A948A8612008A948A961200EC6E0C289F
:10034000E840E8400D6EED501200EC6E0C300D36BA
:10035000E8300D22ED5012000D6A1200EC6E0C40D8
:100360000D6EED501200EC6E0B50030B21DFF4D735
:10037000ECD7E4D7F3D79EA203D09E923BD81100CE
:10038000F2A403D0F2940CD811009EA003D09E904A
:1003900012D81100A1A203D0A19225D81100FF000C
:1003A0008EDF0C740BA802D0B2DF0C820BAA02D035
:1003B000B5DF0C80BAD78EDF0BAE0FD0D8901336D6
:1003C000143606E3EC6E1550131A1650141AED503D
:1003D00002E30C8201D00C9201D00C720BAC02D063
:1003E0009DDF0C80A2D781DF0BAA02D00C9001D038
:1003F0000C709BD7EC6EE85C0022012202220322E3
:10040000ED501200F184EC6E030E9F6E020EA26E90
:10041000880ED56E810ECD6E040ECA6E810EB16E41
:10042000D08E3F0ECB6EED501200EC6E600EF26E71
:10043000ED509E6AEC6E030E9D6EED50A16AEC6E5F
:10044000020EA06EF28EED501200F29A9D6AA06A22
:100450001200F29A12009D901200A09212009D923A
:100460001200F28A12009D801200A08212009D826A
:100470001200C8DFEC6ED70E156EED501368EC6EEF
:10048000500E166EED50146893949396CED7DDD728
:10049000000A04E1ED50000EEC6E010EEF1EFF0AA3
:1004A0001200EC6EF5DFF29E056EEF50046EF28ED8
:1004B000ED50ED501200EC6EEBDFF29E076EEF5048
:1004C000066EF28EED50ED501200EC6EE1DFF29E02
:1004D000096EEF50086EF28EED50ED501200EC6E8A
:1004E0000450EC6E0550DAD7EC6E0650EC6E0750F7
:1004F000D5D7EC6E0850EC6E0950D0D7EC6E310EAB
:100500000B6EFF0ED8DFEC6EFF0EDFD7EC6E210E08
:100510000B6EFF0EDAD7EC6E010E0B6EED50120073
:10052000B2DEBFDFB0DEC7DFAEDECFDFF4D7E46E12
:10053000ED50E46EED501200EC6EE550EC6EE550BF
:100540001200EC6EE3DFF3DFCADFF6DF35D8B4D795
:10055000EC6E830E0B6EFF0EA4DFEC6EFF0EB5DFAC
:10056000EC6E010EA8D7EC6EFF0EEB50EC6EFF0E9A
:10057000EB50120000D8ED50ED501200E46EED503B
:10058000E46EED50ED50E550EC6EE5501200D89061
:10059000EF36E8341200D890E830EF321200800FC6
:1005A000E830400AEF321200E46EED50EDCFE4FF88
:1005B000EF26E550E5201200E46EED50EDCFE4FFAC
:1005C000EF5EE550E5541200E81EEF1E1200E46EE7
:1005D000010EEF26000EE722E5501200E46EFF0E3A
:1005E000EF26E722E5501200EFDFF1D7E46EED5081
:1005F000EDCFE4FF1200FADFEF16E550E51412002C
:10060000F5DFEF1AE550E5181200F0DFEF12E550C4
:10061000E5101200E46EED50ED50E5501200EDCF04
:10062000E4FFEF26000EE5201200EDCFE4FFEF26F9
:10063000FF0EE5201200E8AE01D0F7D7F0D7ED505D
:10064000FF0EEC6EFF0CED50000EEC6E000CED0298
:10065000F4CFE4FFF3CFE4FFED02F450E524E844E7
:10066000010BE52012007FDFF2DFD9D77CDFEFDF5F
:10067000E86CDBD7EC6E320E0B6EED5030DF8BDFAB
:1006800072DF24DF88DF18D70B6A1200EC6E170EBA
:10069000EF60EF6EED50E5DDE4EE7CE1D4D4E2C82E
:1006A0009CBDF7B2ECA8719F7E960C8E13868C7E53
:1006B0007277BE706A6A7164CE5E7C597654B84FA8
:1006C0003F4B06470943463FED50E0DFEC6E1750C5
:1006D00007E0E46EED505FDFE706FDE1E55201D093
:1006E000ED501200ED50176EED501200EEDFDAD62D
:1006F000ECDFE2D6EADFEAD6F2DEED6E1200F4DEDF
:10070000ED6E1200F6DEED6E1200EC6E0B50E46E34
:10071000ED501200EC6EE5500B6EED501200DFDE76
:1007200006D70ADFBFD6E0DE02D706DFC5D6E1DE98
:10073000FED602DFCBD6E9DF0BDFE46EED5000A47E
:1007400001D0FDD700B401D0FDD7E706F8E1E552AE
:10075000E1D7070BD890E834D890E8340109C26E8D
:10076000ED501200C2821200C2A201D0FDD7EC6E81
:10077000C4501200EEDFF6DFF7D7898E1200899E93
:100780001200EC6E1F0E9212929EE10E9312F19ED9
:10079000600EC16E7E0EC06EED50EFD7EC6E000E97
:1007A000E9DF7FDEEC6E010EE5DF85DEEC6E020E2A
:1007B000E1DF8BDEEC6E030EDDDFE00BE844E844A6
:1007C000EC6E7C0E0B16ED500B12040ED3DFE00B1B
:1007D000E844EC6E8F0E0B16ED500B12ED5012002C
:1007E000EC6EF550EC6EF650EC6EF750EC6ED950A6
:1007F000EC6EDA50EC6EFC50EC6EE150EC6EE950B1
:100800001818181A1818E96EED50E16EED50FC6ECC
:10081000ED50DA6EED50D96EED50F76EED50F66E8C
:10082000ED50F56EED501200EC6EF550EC6EF6509A
:10083000EC6EF750EC6ED950EC6EDA50EC6EFC506A
:10084000EC6EE150EC6EE950186E100EFC6EF00E7E
:10085000E16EE00EE96E1950EC6E1A50F3D491DFA0
:0608600008DE9CDFFED75C
:020000040000FA
:020200002ED3FB
:020000040000FA
:02020800B6D06E
:00000001FF
